:100000000C94B8010C94D5010C94D5010C94D50135
:100010000C94D5010C94D5010C94D5010C94D50108
:100020000C94D5010C94D5010C94191F0C94EB1F62
:100030000C940B1A0C94D5010C94D5010C94D50199
:100040000C94D5010C94D5010C94D5010C94D501D8
:100050000C94D5010C94931A0C94D5010C94D501F1
:100060000C94D5010C94D5010C94D5010C94D501B8
:100070000C94D5010C94D5010C94D5010C94D501A8
:100080000C94D5010C94D5010C94D5010C94D50198
:100090000C94D5010C94D5010C94D5010C94D50188
:1000A0000C94D5010C94D5010C94D501DE04DE042A
:1000B0000A050A0572059005A806A8069B053406E0
:1000C0004506450615170B171817601764176417B0
:1000D0006017641764173917641743174D176417AF
:1000E0006417641764176017641764176017641740
:1000F0002617641764175D175D175D175D175D1789
:100100005D175D175D175D176217641715170817E0
:100110006417641764176417641764176417641707
:1001200064176417621764176417601764175B1706
:100130005B175B175B175B175B175B175B175B172F
:10014000621758207F2077217F207721CB20EE2057
:1001500077214521542153005400550056005F007B
:100160006000610057005C005D005E0067005900A0
:100170005A005B003600E200620063005800010094
:100180000100010001004A0052004B000100500034
:1001900000004F0001004D0051004E000100010021
:1001A00049004C0001000100A800AA00A9000100BC
:1001B0000100010001000100010001000100010037
:1001C0000100010001000100010001000100010027
:1001D00004000100005C01000100010001000100B9
:1001E0000100010001000100010001000100010007
:1001F000010001000100100357006F006F00640050
:1002000070006100640000001E0357006F006F0063
:1002100064004B006500790073002E0063006C00E1
:10022000690063006B0000000403090409023B003D
:10023000020100A0FA0904000001030101000921E4
:100240001101000122400007058103080001090493
:100250000100010300000009211101000122B60084
:10026000070582032000011201000200000008EDD2
:10027000FE696001000102000105010902A101857A
:10028000020901A100050919012908150025019598
:1002900008750181020501093009311581257F9515
:1002A000027508810609381581257F950175088139
:1002B00006050C0A38021581257F9501750881060F
:1002C000C0C005010980A101850319012AB70015E5
:1002D0000126B700950175108100C0050C0901A128
:1002E00001850419012AA002150126A002950175B5
:1002F000108100C005010906A1018506050719E066
:1003000029E71500250195087501810205071900E7
:1003100029EF1500250195F07501810205081901E5
:100320002905950575019102950175039101C00597
:10033000010906A101050719E029E7150025019526
:1003400008750181029501750881010507190029C9
:10035000FF150026FF0095067508810005081901A4
:100360002905950575019102950175039101C0005C
:1003700011241FBECFEFDAE0DEBFCDBF11E0A0E059
:10038000B1E0E4E5F4E402C005900D92A438B107B1
:10039000D9F722E0A4E8B1E001C01D92AC38B20761
:1003A000E1F70E9485120C9428220C940000879A91
:1003B0000C94600E8F9A08958F980895CF9383358B
:1003C000910521F0823E910569F143C0FB01C28194
:1003D000CC2371F081E08093860182E00E94F007D7
:1003E000C82F8823B9F183E00E941008C0E032C012
:1003F00083E00E94F00781110FC081E00E94F007A6
:10040000811106C00E94DC0181E00E94100807C033
:100410000E94DA0181E001C083E00E94310810925D
:10042000860118C0FB01C281CC2341F0C091860136
:10043000C111D9CF82E00E9410080CC083E00E9455
:10044000F007882311F083E001C082E00E943108A8
:1004500001C0C1E08C2FCF91089581E008950C94E4
:10046000DE0108950C9431021F93CF93DF9300D0E7
:1004700000D01F92CDB7DEB749835A836B8330918A
:10048000880189819A81311114C0662359F0222391
:1004900049F00E940309182F682F89819A810E94D0
:1004A000AE0803C00E94D808182F69817A81812F75
:1004B00004C00E94030969817A810F900F900F9008
:1004C0000F900F90DF91CF911F910C941C10FC01A5
:1004D000262F408151816281738184810C94340282
:1004E00081E00895CF93DF93EC0160E00E94670202
:1004F000BE01DF91CF910C9432020C9449110C94FF
:10050000451108950E9438070E9481022FEF84E36D
:100510009CE0215080409040E1F700C000000C9426
:10052000B91A0F931F93CF93DF938C0161E00E9460
:100530006702EC01B8010E942F028823F1F1B80193
:10054000CE010E9457188823C1F1B801CE010E9444
:100550001B15882391F1B801CE010E94B31788239F
:1005600061F1F8018281882309F1CB358DE5D80747
:10057000C1F050F4C115FCE5DF0781F0CF3DDC454B
:10058000A9F40E94340E19C0CC35EDE5DE0761F008
:10059000CD35DD4559F40E947D0D08C00E948202D0
:1005A0000CC00E94860D02C00E94890DC801DF9117
:1005B000CF911F910F910C942D0280E0DF91CF918C
:1005C0001F910F9108950E94EE190C94FC020E9455
:1005D000FF020C94F41908950C94EB0281E0089545
:1005E0000C94EE020895CF93C82F0E94EC028C2F3A
:1005F0000E94F002CF91089580E00C94F3020E94D3
:10060000B3180C94F3020E94B318909187018917D4
:1006100021F0809387010C94F3020895CF93DF9328
:10062000CDB7DEB72B970FB6F894DEBF0FBECDBFA8
:100630004F83588769877A878B8761110E94C90C1D
:100640009E012F5F3F4F86E0F90111928A95E9F7ED
:1006500085E0FE013796D90101900D928A95E1F768
:1006600089819A814C815D81452B31F09F3F31F426
:1006700091E08F3F19F403C091E001C090E090FF3A
:1006800009C049815A816B817C818D819E810E9444
:10069000EA0B05C0C9010E9470028111F2CF2B96AE
:1006A0000FB6F894DEBF0FBECDBFDF91CF91089596
:1006B000FC01808191810E9445090895CF93882390
:1006C00009F4A9C0C82F8238C1F40E94B31881FD73
:1006D000A2C069E380910201909103010E94A919CF
:1006E0000E94EB0C2FEF81EE94E02150804090406F
:1006F000E1F700C0000069E319C0833801F50E94EA
:10070000B31880FD88C063E58091020190910301D8
:100710000E94A9190E94EB0C2FEF81EE94E021506A
:1007200080409040E1F700C0000063E58091020145
:10073000909103010E94B419CF910C94EB0C843872
:10074000C1F40E94B31882FD66C067E48091020183
:10075000909103010E94A9190E94EB0C2FEF81EEEA
:1007600094E0215080409040E1F700C0000067E431
:10077000DDCF8CEF8C0F813AF8F48C2F0E946A1732
:10078000811149C06C2F80910201909103010E9458
:100790002919882349F06C2F80910201909103015F
:1007A0000E94B4190E94EB0C6C2F80910201909171
:1007B00003010E94A919C0CF80E28C0F883048F451
:1007C000C77081E001C0880FCA95EAF70E94AC0C9F
:1007D000B3CFEBE5EC0FE33040F4F0E0E95BFE4F24
:1007E000808190E0CF910C94E718E8E5EC0FE731B9
:1007F00050F4F0E0EE0FFF1FE75EFE4F8081918125
:10080000CF910C94FD18CD3E30F08C2F0E940A132E
:10081000CF910C94DC13CF910895882309F464C020
:10082000823879F40E94B31881FF5EC069E3809139
:100830000201909103010E94A9190E94EB0C69E347
:1008400010C08338B1F40E94B31880FF4DC063E537
:1008500080910201909103010E94A9190E94EB0C62
:1008600063E580910201909103010E94B4190C94F8
:10087000EB0C843879F40E94B31882FF35C067E42A
:1008800080910201909103010E94A9190E94EB0C32
:1008900067E4E7CF9CEF980F913A10F4682FE1CF0F
:1008A00090E2980F983050F4877091E001C0990F52
:1008B0008A95EAF7892F0E94B20CD9CF9BE5980F51
:1008C000933020F480E090E00C94E71898E5980FBE
:1008D000973120F480E090E00C94FD188D3E20F0DC
:1008E0000E9465130C94DC1308951F93CF93DF933C
:1008F000182FEB010E945E03209741F08FE99FE0E3
:100900000197F1F700C000002197F6CF812FDF910A
:10091000CF911F910C940D04893319F060E070E0C1
:1009200002C060E570E00C947504882321F00E94F9
:10093000AC0C0C94EB0C0895882321F00E94B20CAF
:100940000C94EB0C0895CF92DF92EF92FF920F93ED
:100950001F93CF93DF937C01D62FC72FFC01128109
:10096000058102950F700E94A20C8823B9F0112313
:10097000A9F08C2F807F803421F080E28D0F8830A9
:1009800068F08091700282FD09C082E00E944B0DE8
:100990000E94A20C91E0D82ED92601C0D12CCC2ED9
:1009A000C2948FE0C8228C2D90E08C30910508F025
:1009B000CFC1FC01EA5AFF4F0C94BF218C2F807FDE
:1009C000CF70882311F0C295C07F112399F0CC23FA
:1009D00009F4AAC180E28D0F883010F0D11104C053
:1009E0008C2F0E94AC0C03C08C2F0E94BC0C0E9468
:1009F000EB0C9AC18D2F0E940D04CC2309F4A8C1E1
:100A000080E28D0F883038F1DD2329F18C2F0E9490
:100A1000C20C24C08C2F807FCF70803211F0C29521
:100A2000C07FDD2319F0D130A1F13DC0809170026B
:100A300082FF17C0112349F0CC2329F08C2F0E948C
:100A4000AC0C0E94EB0C80E070C180E00E940D04B1
:100A5000CC2309F47DC18C2F0E94B20C0E94EB0CB8
:100A600077C1112371F0002341F0013031F40E946D
:100A7000CC0C8C2B0E94D40C6BC10E94CC0C8C2B08
:100A80001DC0002319F0013009F462C10E94E10C7D
:100A900025C0112321F0063008F05AC10EC00530E0
:100AA00008F056C11BC0112361F0002331F0F7019B
:100AB000858180FF39C18F7085838C2F0E949504BA
:100AC00047C1002359F0D93309F03FC1FFEF07EECA
:100AD00013E0F15000401040E1F735C18C2F0E9427
:100AE0009C0436C18C2F86958695837019F08130D1
:100AF00061F02EC1112321F08D2F9C2F937002C025
:100B000080E090E00E94E7182BC1112321F08D2F87
:100B10009C2F937002C080E090E00E94FD1820C1DD
:100B20008D2F112319F00E940A1302C00E94651331
:100B30000E94DC1315C18C2F837009F047C011117E
:100B40000BC12D2F229526952770220F220F6D2F76
:100B50006F70862F90E0A0E0B0E0022E04C0880FF6
:100B6000991FAA1FBB1F0A94D2F7D4FF10C04FE0F1
:100B700050E060E070E004C0440F551F661F771F0F
:100B80002A95D2F7409550956095709503C040E046
:100B900050E0BA01C695C695C3708A019B01082B27
:100BA000192B2A2B3B2BC901B801C23049F058F44C
:100BB000C13019F00E94A407CFC00E949207CCC098
:100BC0000E94B607C9C00E949007C6C0112319F041
:100BD0008C2F817001C08695882309F4BDC02D2F0C
:100BE000229526952770220F220F6D2F6F70862F6A
:100BF00090E0A0E0B0E0022E04C0880F991FAA1F69
:100C0000BB1F0A94D2F7D4FF10C04FE050E060E061
:100C100070E004C0440F551F661F771F2A95D2F756
:100C2000409550956095709503C040E050E0BA0142
:100C3000C695C695C3708A019B01082B192B2A2BD8
:100C40003B2BC901B801C23049F058F4C13019F04A
:100C50000E94890881C00E9477087EC00E949B087C
:100C60007BC00E94CA0778C0CF70112339F08C2F47
:100C70000E9410088D2F0E9495046EC08D2F0E9437
:100C80009C048C2F0E94310867C0D23F21F128F4C8
:100C9000D03F41F0D13FC1F043C0D33F19F1D43F21
:100CA00079F03EC0112341F0053008F051C08C2F7F
:100CB0008F710E9456084CC0063008F049C0F7CF2B
:100CC0008091700282FF18C0112339F08C2F8F7130
:100CD0000E9410083DC01123C9F38C2F8F710E9410
:100CE000310836C0112329F08C2F8F710E94FB0729
:100CF0002FC00E94D6072CC0112349F0CF718C2F32
:100D00000E94100863E08C2F0E94300D21C081E00A
:100D10000E944B0D0230E0F082E00E944B0D18C0A3
:100D2000112331F0002391F28D2F0E945E0310C039
:100D3000002399F2D93349F41FEF27EE33E0115025
:100D400020403040E1F700C000008D2F0E940D04CC
:100D500088EF8C0D843020F40E94B3180E94F302B7
:100D6000DD20C9F00E949E0C80FD15C0F7011282A3
:100D70000E94980C0E941008C7010E94EC060E9475
:100D8000980CDF91CF911F910F91FF90EF90DF9022
:100D9000CF900C943108DF91CF911F910F91FF906C
:100DA000EF90DF90CF9008950F931F93CF93DF9331
:100DB000EC01688179818A810E9450098C010E942E
:100DC000AD080E947E07B801CE010E94A304DF9106
:100DD000CF911F910F910895CF93DF93EC019881EC
:100DE00089812B813C81232B31F08F3F31F481E0CD
:100DF0009F3F19F403C081E001C080E080FD1DC069
:100E0000CE010E949102811110C00E94A20C882381
:100E1000A1F08A81882389F08091700282FD0DC043
:100E200082E0DF91CF910C944B0DCE010E94D4064D
:100E3000CE01DF91CF910C947202DF91CF91089592
:100E400080E090E00E94E71880E090E00E94FD18AA
:100E50000E94C90C0E94EB0C0E940D150C94DC132F
:100E600080910201909103010E94BF190C94200708
:100E70000E94B90C0C94300792959F70963079F0CF
:100E800010F4925001C09A50923068F4803F69F09B
:100E900018F4883E40F409C0843F29F406C0883E17
:100EA00020F0813F11F080E0089581E00895FC0179
:100EB000808191810E9445090E943C070895CF934B
:100EC000DF9300D000D01F92CDB7DEB70F900F9008
:100ED0000F900F900F90DF91CF910895CF93DF93F4
:100EE00000D000D000D0CDB7DEB726960FB6F8946C
:100EF000DEBF0FBECDBFDF91CF9108950895089555
:100F00000C947F070C9480070E94820760939C01D9
:100F100070939D0180939E0190939F010C942007F4
:100F20000C9484070F931F9300919C0110919D01D5
:100F300020919E0130919F01602B712B822B932B6E
:100F40001F910F910C9484070F931F9300919C01A4
:100F500010919D0120919E0130919F01602371238A
:100F6000822393231F910F910C9484070F931F9357
:100F700000919C0110919D0120919E0130919F0153
:100F800060277127822793271F910F910C94840764
:100F90000C947F070E94C807609398017093990191
:100FA00080939A0190939B010C94200760E070E07D
:100FB000CB010C94CA07611571058105910529F4CF
:100FC00081E0442361F080E00895DC01CB0104C09E
:100FD000B695A795979587954A95D2F7817008950C
:100FE000482F609198017091990180919A01909198
:100FF0009B010C94DB070F931F9341E050E060E0EE
:1010000070E08A019B0104C0000F111F221F331FD3
:101010008A95D2F7C901B8011F910F910C94CA07A4
:101020000F931F9341E050E060E070E004C0440F74
:10103000551F661F771F8A95D2F78091980190916E
:101040009901A0919A01B0919B018A019B01082B03
:10105000192B2A2B3B2BC901B8011F910F910C941E
:10106000CA070F931F9341E050E060E070E004C0B6
:10107000440F551F661F771F8A95D2F740955095EC
:10108000609570958091980190919901A0919A0135
:10109000B0919B018A019B01082319232A233B233A
:1010A000C901B8011F910F910C94CA070F931F93A8
:1010B00041E050E060E070E004C0440F551F661F3F
:1010C000771F8A95D2F78091980190919901A0910C
:1010D0009A01B0919B018A019B01082719272A27B1
:1010E0003B27C901B8011F910F910C94CA070F93B8
:1010F0001F93009198011091990120919A013091CC
:101100009B01602B712B822B932B1F910F910C94C1
:10111000CA070F931F930091980110919901209194
:101120009A0130919B0160237123822393231F91A5
:101130000F910C94CA070F931F930091980110917F
:10114000990120919A0130919B0160277127822794
:1011500093271F910F910C94CA070895990F990F27
:10116000890FE82FE695E695E695877051E001C076
:10117000550F8A95EAF785E0E89FF0011124E757BB
:10118000FE4F20E030E070E04081CB01022E02C033
:10119000969587950A94E2F7817081958427852337
:1011A000842781932F5F3F4F2530310569F70895DC
:1011B000990F990F890F682F669566956695982FF8
:1011C000977085E0689FB001112440E050E080E016
:1011D000FB01E40FF51FE757FE4F208130E0092E99
:1011E00002C0369527950A94E2F721703327042E22
:1011F00001C0220F0A94EAF7822B4F5F5F4F453000
:10120000510531F70895BF92CF92DF92EF92FF928E
:101210000F931F93CF93DF938C01C0909801D090D0
:101220009901E0909A01F0909B0180919C0190912E
:101230009D01A0919E01B0919F01C82AD92AEA2A56
:10124000FB2ACFE1D0E0D701C6010C2E04C0B69531
:10125000A795979587950A94D2F780FD04C02197AA
:1012600090F7B12C07C0BC2EB8018C2F0E94301013
:101270000197A9F38B2DDF91CF911F910F91FF90D3
:10128000EF90DF90CF90BF900895CF93DF93EC0164
:101290000E940309BE010E943010DF91CF91089592
:1012A0001F93CF93DF93EB0190918801992321F055
:1012B000CB010E94450913C0882349F0CB010E944D
:1012C0000309182F682FCE010E94AE0804C0CB017D
:1012D0000E94D808182FBE01812F0E943010DF9184
:1012E000CF911F9108951F93CF93DF93C091A001D9
:1012F00016E08091A101C81799F0D0E01C9FF00181
:101300001D9FF00D1124EE55FE4F408151816281E9
:101310007381848195810E946E072196C770E9CF01
:10132000DF91CF911F9108954091D2015091D30147
:101330006091D4017091D5018091D6019091D7012F
:101340000C946E07EF92FF920F931F93CF93DF934E
:101350008091D70182958F7009F065C08091D4018A
:10136000882309F460C08091A001F090A101109140
:10137000D2010091D3016091D5017091D60191E025
:101380001F3F09F090E0C0910001D0910101292F89
:1013900096E0E92E8F1509F446C06115710521F01C
:1013A0000F3F21F030E003C031E001C0322F90E068
:1013B00030FD36C0E89EF001E99EF00D1124DF01FA
:1013C000AE55BE4F11963C911197301329C03C91F8
:1013D000311326C012963C911297311121C01396F9
:1013E0004D915C911497461B570B4C175D07C0F449
:1013F0008091D7018F7080618093D701E955FE4FAE
:1014000080818F708061808382ED91E00E94EC0684
:10141000DF91CF911F910F91FF90EF900C94730982
:1014200001968770B7CFDF91CF911F910F91FF90F9
:10143000EF9008959F92AF92BF92CF92DF92EF927A
:10144000FF920F931F93CF93DF93CDB7DEB76197D2
:101450000FB6F894DEBF0FBECDBF8C0185E0F8015A
:10146000DE011D9601900D928A95E1F7D801129642
:10147000EC909091D201E091D3012091D50130916F
:10148000D6012115310531F0EF3F31F481E09F3F66
:1014900019F403C081E001C080E0B82FB1709B2E29
:1014A00080FD47C1D8014C9111965C91119713961C
:1014B000AD90BC90149782EDC82E81E0D82EF090AC
:1014C000D401B501621B730B209100013091010121
:1014D000FF2009F4D9C08091D7016217730708F083
:1014E00095C0282F207F09F052C05E1313C0491306
:1014F00011C0FE2CE1100EC08F7080618093D70167
:101500000E949409C6010E94EC068091D701F8015F
:1015100085834DC1AB2831F05F3F31F481E04F3F0F
:1015200019F403C081E001C080E080FD03C081E0C8
:101530008E2502C080E090E0F82FF170FF2E80FF32
:101540001CC08091A0012091A10136E0821709F40E
:101550000BC190E0389FF001399FF00D1124EE553A
:10156000FE4F6181561306C06081461303C062813D
:10157000E61203C001968770E9CFFE2CEE2009F435
:1015800016C18091D70181608093D70154C05E134A
:1015900006C0491304C0E11002C0F80199C0C80197
:1015A0000E945707882361F1EE2051F12091D70165
:1015B000822F82958F7090E0029774F08091D20113
:1015C0009091D30198878F831986BB86AA862C8732
:1015D000CE0107960E94EC0686E0F801A2EDB1E08C
:1015E00001900D928A95E1F70E94A2090E94940948
:1015F0000AC05E1711F1C8010E94570781112CC063
:10160000C8010E94EC06FF24F394D1C0282F207F4C
:1016100081F77A2DB98AA88A6E2D89890E945F0781
:1016200082ED91E00E94EC0686E0D6011D928A953B
:10163000E9F70E949409F12CBAC04913DCCFE110FC
:10164000DACFF8018583C8010E94EC0686E0D60156
:101650001D928A95E9F7ABC0EE2091F22091D70157
:10166000822F82958F7090E002970CF4B5CF809115
:10167000D2019091D3019A8389831B82BD82AC826F
:101680002E83CE010196A6CF6217730708F044C0DF
:10169000FE2CEE2009F4B4CF5E1330C049132EC0E7
:1016A0002091D70120FD21C0822F82958F70482F75
:1016B00050E041155105C9F0F80125834F3051051F
:1016C00041F08F5F982F9295907F822F8F70892B9A
:1016D0008583C8010E94EC0686E0F801A2EDB1E026
:1016E00001900D928A95E1F73CC086E0F801A2EDE9
:1016F000B1E001900D928A95E1F759C0C8010E94AE
:101700005707811169CF8091D70181608093D701FC
:10171000C8010E94EC064BC07A2DB98AA88A6E2DAA
:1017200089890E945F0786E0D6011D928A95E9F7B4
:1017300018C0EE2009F464CFC8010E945707F82EA4
:10174000882309F45DCF86E0F801A2EDB1E00190B5
:101750000D928A95E1F782ED91E00E9458030E9474
:10176000A2090E94940923C04D875E878D859E85BE
:101770000E944509292F22952F70223028F49F704E
:1017800039F0811105C00BC0243028F49F7049F452
:10179000805E883020F0C8010E94EC069F2CF92C56
:1017A00006C0D80115969C91907F91F7F8CF8F2DA8
:1017B00061960FB6F894DEBF0FBECDBFDF91CF911B
:1017C0001F910F91FF90EF90DF90CF90BF90AF905F
:1017D0009F9008951F93CF93DF93CDB7DEB72C97DB
:1017E0000FB6F894DEBF0FBECDBF4F835887698711
:1017F0007A878B879C87CE0107960E941A0A8823D6
:10180000D1F09F8188852A853B85232B31F08F3F3E
:1018100031F481E09F3F19F403C081E001C080E012
:1018200080FD47C04F81588569857A858B859C8569
:101830000E946E073EC086E0FE013796DE011196DB
:1018400001900D928A95E1F7FF81E8856A857B8595
:101850006115710531F0EF3F31F481E0FF3F19F47C
:1018600003C081E001C080E080FD23C02091A10180
:1018700030E0C9010196877099274091A00150E09E
:1018800084179507F1F1F983EA837D836C8396E0F1
:10189000929FD001939FB00D1124AE55BE4FFE0113
:1018A000319601900D929A95E1F78093A1010E94E3
:1018B000730916E08091A0019091A101891771F13F
:1018C000189FC00111248E559E4F0E941A0A88232A
:1018D00029F1E091A0011E9FF0011124EE55FE4F69
:1018E0004081518162817381848195810E946E075C
:1018F0008091A00190E00196877099278093A001C4
:10190000D9CF0E9438071092A1011092A001E2EDF8
:10191000F1E086E0DF011D928A95E9F72C960FB67B
:10192000F894DEBF0FBECDBFDF91CF911F91089518
:101930008091F80185958595859508958091F801A8
:10194000877008959091F801977081E009F480E024
:10195000089580911B02089590911B02892B80931A
:101960001B020895809590911B02892380931B028E
:10197000089510921B02089590911A02892B80936A
:101980001A020895809590911A02892380931A0271
:10199000089510921A0208958091F901089508950A
:1019A0000C94CF0C0C94D00C9091700292FD08C056
:1019B0009091F901981721F08093F9010C94D20CC1
:1019C00008958091F901882329F01092F90180E0AF
:1019D0000C94D20C0895CF93DF93E0910201F09123
:1019E000030180911B028083E0910201F0910301C9
:1019F000908180911A02892B80838091F90188233C
:101A000081F0E0910201F09103019081892B8083A4
:101A100080910201909103010E94131981110E948B
:101A2000E10CC0910201D091030140E250E068ED69
:101A300071E0CE010E94D921892B69F080E2FE017C
:101A4000A8EDB1E001900D928A95E1F7CE01DF910A
:101A5000CF910C94BF18DF91CF9108950C94CF0CC7
:101A60009091700292FD10C098E0899F900111241E
:101A7000262B2093F8010E9410088091F80185958B
:101A8000859585950C942E0D0C9410081092F801F4
:101A900080E00C942E0D2091F80180958223809394
:101AA000F801982F977099F430E0482F082E000C19
:101AB000550B2417350759F09091700292FD07C01D
:101AC0008595859585950E9431080C94460D08955D
:101AD0009091700292FB222720F9281769F080FB71
:101AE00092F99093700280916F02909170020E941F
:101AF000B00D82E00C944B0D08958091700282FB32
:101B0000882780F991E089270C94680D81E00C9476
:101B1000680D80E00C94680D80E090E00E94EE215A
:101B200021E0893E9E4F09F020E0822F089582E057
:101B300090E00C94E62183E090E00C94E621CF93B2
:101B400084E090E00E94E621C82F82E290E00E94AB
:101B5000E6212C2F30E0A901582BCA01CF9108951E
:101B6000CF93C92F682F84E090E00E94F4216C2F5E
:101B700082E290E0CF910C94F421AB01BC018FE0A4
:101B800090E00C940622AB01BC0183E190E00C9440
:101B9000062260E070E0CB010C94C30D60E070E0C1
:101BA000CB010E94BD0D0C94C90D69EE7EEF80E063
:101BB00090E00E94122260E082E090E00E94F42116
:101BC00060E083E090E00E94F42110929C0110926A
:101BD0009D0110929E0110929F0160E084E090E0D0
:101BE0000E94F42160E082E290E00E94F42160E033
:101BF00085E090E00E94F42160E086E090E00E94A1
:101C0000F4216FEF87E090E00E94F42140E050E083
:101C1000BA0188E090E00E94062260E08DE090E04A
:101C20000E94F42140E050E0BA0188E190E00E9477
:101C3000062260E087E190E00E94F42140E050E05D
:101C4000BA018CE190E00E94062260E070E080E240
:101C500090E00E94122240E050E0BA0188E190E05A
:101C60000E9406220C94CE0D0C94D50D682F8EE0A8
:101C700090E00C94F4210E94781A609325027093EE
:101C8000260280932702909328026093210270938A
:101C900022028093230290932402089585B78068DE
:101CA00085BF85B7806885BF089581E008950C944D
:101CB000550E08950C94590E0C94590E0C945C0E0C
:101CC0000C94590E0C94590E0E944E0E8CE091E12A
:101CD0000E94A9180E94620E0C94D7010E945A0E0D
:101CE0000C94590E0E940F110C94F2020E94631A78
:101CF0000E94E6110E94720E0C945E0E8F929F92CB
:101D0000AF92BF92CF92DF92EF92FF920F931F9309
:101D1000CF93DF93CDB7DEB72A970FB6F894DEBF27
:101D20000FBECDBF0E94FB11982E81110E943B0E69
:101D30008CE1A82E82E0B82E00E010E0802E802FEB
:101D40000E943311D82EF501C1905F01C826B1F46D
:101D50000F5F1F4F0530110589F78FEF89838A8345
:101D60001B820E946C1A8160782F9D838C8349812D
:101D70005A816B818D810E940E032FC080912902B0
:101D800081FD0E943911E12CFF24F3948C2D8F21C9
:101D9000F1F00E94570E882399F0EE828F82DF20A7
:101DA00081E009F480E088870E946C1A8160782FB6
:101DB0009A8789874E815F8168858A850E940E0394
:101DC000F801E45EFD4F8081F826F08206C0E394BE
:101DD000FF0CF4E0EF12DACFBBCF81E0911001C02D
:101DE00080E02A960FB6F894DEBF0FBECDBFDF911C
:101DF000CF911F910F91FF90EF90DF90CF90BF9008
:101E0000AF909F908F9008950E947E0E0E94FA13CB
:101E10000C940303CF93DF930E943510EC018115DE
:101E200021E5920708F045C0811530E5930708F0D9
:101E300094C0883E910528F5803E910508F0F8C0D1
:101E4000883A910570F4853A910508F07CC081309C
:101E5000910509F475C008F4E8C0049708F0E8C0DB
:101E6000E4C08F3B910508F0E0C0C85AD0E0CC0F29
:101E7000DD1FC65BDE4F0990D881C02DCE01946472
:101E8000D8C0811540E2940758F4811551E09507B8
:101E900008F0CEC08D3E910508F4C7C09065C9C05A
:101EA000C11580E4D80708F4C0C0DF70CE01906A85
:101EB000C0C0811525E59207A8F4811534E5930784
:101EC00008F095C0811543E5940708F07BC08115A3
:101ED00052E5950708F061C0D82FCC27CE01816F5D
:101EE000906AA7C0C11589E5D807A0F4C11528E5F7
:101EF000D20708F082C0C11536E5D30708F095C0B7
:101F00008C2F0E94C9108F7190E0D82FCC27CE0162
:101F100090628FC0C1154AE5D40708F474C0CE01A1
:101F200090568115904208F080C08D2F8F710E94CD
:101F3000C910DD27D0628F71AE01582BCA0179C05C
:101F400081E090E076C0C55AD0E0C858DE4F888165
:101F5000C82FD0E0CE0190646CC074E09695879550
:101F60007A95E1F7282F23703C2F337081E090E0C1
:101F700002C0880F991F3A95E2F79C68AC01522B7A
:101F80009A019C2F9F709695969550E2959FE0013F
:101F90001124C9018C2B9D2B4CC08370992721E003
:101FA00030E002C0220F331F8A95E2F79C2F9695EE
:101FB000969580E2989FE0011124C22BD32BCE018D
:101FC0009C6837C08370992721E030E002C0220F5F
:101FD000331F8A95E2F79C2F9695969540E2949F41
:101FE000E0011124C22BD32BCE019A6822C0D82F36
:101FF000CC27CE01846F906A1CC0DC2FCC27CE0189
:10200000806F906A16C08C2F8F700E94C91094E068
:10201000D695C7959A95E1F7CF70D0E0DC2FCC2705
:10202000D0699E01282BC90104C080E090E001C066
:10203000CE01DF91CF910895E72FF0E095E0899FE1
:10204000E00DF11D1124EE0FFF1FEE0FFF1FE60F35
:10205000F11DEE0FFF1FEA5AFE4F859194910895EE
:102060000E941C100E940A0F08958238910569F1A0
:10207000B0F48133910509F46DC048F489329105BB
:1020800009F463C08A32910509F469C00895853363
:10209000910509F455C089339105B9F00895833E3F
:1020A000910569F138F4803E9105B1F0823E9105C9
:1020B00009F10895863E9105A9F1873E9105B9F190
:1020C000843E910509F064C023C020916F0220FD79
:1020D0004FC021FD4DC0089580916F0280FD44C026
:1020E0008091700280FF44C080916F0284FD42C0E5
:1020F00083EE4DC080916F0282FF38C0F5CF809192
:102100006F0282FD33C08091700280FD31C0ECCF40
:102110008091700281FF32C080916F0284FD2AC0DD
:1021200087EE35C080916F0283FF26C0F5CF809186
:102130006F0283FD21C08091700281FD1FC0ECCF32
:1021400080916F0285FD1CC01DC080916F0285FDCE
:1021500019C016C080916F0286FD16C017C080910D
:102160006F0286FD13C010C089E311C082EE0FC05C
:1021700080EE0DC080E00BC086EE09C084EE07C083
:1021800089E205C085E303C08AE201C081E390E0F3
:10219000089590916F0292FF0DC0282F287128306A
:1021A00019F4877F846006C0282F2471243011F42D
:1021B0008B7F886093FF0DC0282F2871283119F478
:1021C000877E846106C0282F2471243111F48B7E10
:1021D00088612091700220FF0DC0382F387138308F
:1021E00019F4877F816006C0382F3171313011F4C6
:1021F0008E7F886021FF0DC0282F2871283119F4A7
:10220000877E816106C0282F2171213111F48E7ED5
:10221000886194FD877E089580E0089508950E9466
:102220008C0D811102C00E94340E0E94970D809384
:1022300029020E949F0D9093700280936F020E946A
:102240000E110E949B0D682F70E080E090E00E94CC
:102250009007609198017091990180919A019091F5
:102260009B010C94C807E82FF0E0EA58FD4F8081ED
:102270000895089580EA8A95F1F7089500C00895B9
:102280000C943A1108950C9442110C9443110C943F
:1022900042110C944711F894E82FE295EF70F0E0AA
:1022A00031A1282F2F7081E090E001C0880F2A957E
:1022B000EAF7982F9095932391A392A1892B82A35B
:1022C000789408950F931F93CF93DF93CFE7D1E0D6
:1022D00089918F3F11F00E944B1181E0C438D807DB
:1022E000B9F7CBE7D1E00FE711E089918F3F11F00B
:1022F0000E944B110C171D07C1F7DF91CF911F9161
:102300000F910895CF92DF92EF92FF920F931F9358
:10231000CF93DF938C01C62FD0E0CE0181589E4F22
:102320007C01FC0190819F3F09F447C0D62EF894B0
:10233000E92FE295EF70F0E081A19F7021E030E09D
:1023400001C0220F9A95EAF7822B81A382A12095E2
:10235000282322A378940E943E11EBE7F1E04FE797
:1023600051E031E0C12C21912F3F89F0A22FA2959D
:10237000AF70B0E090968C9190E02F7002C0959570
:1023800087952A95E2F780FD02C0832F01C080E087
:10239000C82A330F4E175F0731F7F70180818F3F4F
:1023A00011F00E944B1161E0C11001C060E08D2D61
:1023B0000E944011C00FD11FC882DF91CF911F91A1
:1023C0000F91FF90EF90DF90CF9008950E946211DF
:1023D00085E0E6E7F2E0DF01982F1D929A95E9F794
:1023E000E1E7F2E0DF011D928A95E9F785E00E94BE
:1023F00042120C947D02FF920F931F93CF93DF93B1
:1024000000D000D01F92CDB7DEB78E010F5F1F4FF7
:1024100085E0F80111928A95E9F7F12C6F2DC8013A
:102420000E948211F394F5E0FF12F8CF45E050E0EE
:10243000B80181E792E00E94D921FF24F39400972C
:1024400009F4F12C892B41F085E0F801A1E7B2E015
:1024500001900D928A95E1F72F2D45E066E772E035
:1024600081E792E00E9443120E947F028F2D0F901D
:102470000F900F900F900F90DF91CF911F910F91C0
:10248000FF9008950895FF920F931F93CF93DF93CA
:102490008C01F62ED72FC42F222349F081E08093A0
:1024A0002C020E946C1A90932B0280932A02809136
:1024B0002C028823C1F080912A0290912B020E9465
:1024C000841A059780F0EF2DFD2FD8014C2F50E096
:1024D000CD01801B910B841795071CF48D9181937E
:1024E000F7CF10922C02DF91CF911F910F91FF90A7
:1024F00008950E94711C0E94760E0C947D1C0E940F
:10250000811C0E94040F0C949B1C0E940A1A0E94BA
:10251000581C0E94640E0E9479120E947F120E9431
:102520006E0EFBCF8091330280FF06C060910901DF
:1025300070E0660F771F26C081FF04C0609109011B
:1025400084E005C082FF07C06091090188E0689FB0
:10255000B001112417C0909132029923D1F06091FB
:102560000801961788F72091090188E0289F9001BB
:102570001124929FA001939F500D112470E0CA0175
:102580000E94AB216038710540F46115710519F4A2
:1025900006C068E070E0862F08958FE7089581E017
:1025A00008958091330280FF08C06091050170E0BA
:1025B000759567957595679521C081FF06C06091F7
:1025C000050170E07595679519C082FF04C06091A0
:1025D000050170E010C090913102992399F060914B
:1025E00004019617A0F780910501899FC00111246D
:1025F00070E00E94AB216038710540F461157105EF
:1026000019F406C061E070E0862F08958FE7089501
:1026100081E008958D3E21F40E949212819504C0BC
:102620008E3E29F40E9492128093370208958F3EC5
:1026300021F40E949212819504C0803F29F40E94E7
:102640009212809336020895893F19F40E94D112A4
:1026500005C08A3F31F40E94D112819580933802DF
:1026600008958B3F21F40E94D112819504C08C3FC4
:1026700029F40E94D1128093390208959FE0980FA7
:10268000983078F421E030E0A90102C0440F551FD2
:102690009A95E2F7CA0190913502892B8093350211
:1026A00008958D3F21F48091330281600BC08E3FED
:1026B00021F480913302826005C08F3F29F480911C
:1026C000330284608093330208958D3E39F49091F3
:1026D000370297FF35C01092370259C08E3E29F459
:1026E000909137021916BCF32BC0909136028F3EA1
:1026F00029F497FF25C01092360249C0803F19F493
:102700001916CCF31DC090913802893F29F419168F
:10271000BCF4109238023BC08A3F19F497FF10C0F6
:10272000F8CF8B3F39F49091390297FF09C010928E
:1027300039022DC08C3F21F4909139021916BCF357
:102740009FE0980F983080F421E030E0A90102C0AA
:10275000440F551F9A95E2F7CA0180959091350272
:1027600089238093350213C08D3F21F48091330279
:102770008E7F0BC08E3F21F4809133028D7F05C088
:102780008F3F29F4809133028B7F809333028091B5
:102790003602811106C080913702811102C0109269
:1027A000320280913802811106C080913902811174
:1027B00002C01092310208950E946C1A20913602D4
:1027C000211104C020913702222321F0909330027E
:1027D00080932F0220913802211104C020913902E8
:1027E000222321F090932E0280932D0284E392E025
:1027F0000C94D918EF92FF920F931F93CF93DF930E
:1028000000D000D000D0CDB7DEB786E0E4E3F2E040
:10281000DE01119601900D928A95E1F7E090360263
:10282000F09037020091380210913902109236026E
:10283000109237021092380210923902E11003C050
:10284000FF2009F45DC080912F02909130020E9418
:10285000841AAC0190913202992339F020910A0137
:1028600030E02417350758F04BC020910B018AE067
:10287000289F900111242417350718F041C09F3F6D
:1028800019F09F5F90933202EE2061F00E94921245
:102890001E1414F09FEF01C091E0989F902D112419
:1028A00090933602FF2061F00E9492121F1414F0E0
:1028B0009FEF01C091E0989F902D112490933702D3
:1028C000309136023323E1F0209137022223C1F008
:1028D00045EB3403C0011124992319F0909336027B
:1028E00003C081E08093360235EB2303C00111243D
:1028F000992319F09093370203C081E08093370247
:10290000011103C0112309F45DC080912D02909143
:102910002E020E94841AAC0190913102992339F061
:102920002091060130E02417350758F04BC0209164
:1029300007018AE0289F900111242417350718F019
:1029400041C09F3F19F09F5F90933102002361F0D7
:102950000E94D112101614F09FEF01C091E0989FD1
:10296000902D112490933802112361F00E94D1120E
:10297000111614F09FEF01C091E0989F902D112443
:1029800090933902309138023323E1F020913902DB
:102990002223C1F045EB3403C0011124992319F01F
:1029A0009093380203C081E08093380235EB230313
:1029B000C0011124992319F09093390203C081E0DA
:1029C000809339028091360281110BC080913702C9
:1029D000811107C080913802811103C080913902B2
:1029E00081110E94DC13EB82FC820D831E8386E042
:1029F000FE013196A4E3B2E001900D928A95E1F7D1
:102A000026960FB6F894DEBF0FBECDBFDF91CF91F3
:102A10001F910F91FF90EF900895E4E3F2E086E0BC
:102A2000DF011D928A95E9F710923202109231026D
:102A3000109233020895CF93DF93EC01FB01828162
:102A4000882309F43CC1C430FDE5DF0760F4CB3FC7
:102A50009CE5D90788F49E0122503C45243131057C
:102A600008F02EC109C0C236EDE5DE0729F0C63AEE
:102A7000FDE5DF0709F024C10E949F0D90937002CD
:102A800080936F02C1318CE5D80709F4C6C008F005
:102A900042C0C930ECE5DE0709F49BC000F5C53043
:102AA0008CE5D80709F485C078F4C330ECE5DE077F
:102AB00009F478C008F07AC0C230DC4509F0F5C0EE
:102AC00080916F028160EFC0C7309CE5D90709F49F
:102AD00078C008F07AC080916F028061E4C0CD3088
:102AE000FCE5DF0709F487C058F4CB309CE5D90733
:102AF00009F479C008F07BC080916F0288606FC0D4
:102B0000CF30FCE5DF0709F480C008F082C0809177
:102B10006F02877FC8C0CE3F9CE5D90709F471C01A
:102B200000F5C531FCE5DF0709F485C068F4C33161
:102B30009CE5D90709F475C008F095C00E943807D4
:102B400080916F028F77AFC0CC3FFCE5DF07A9F122
:102B500008F054C0CB3FDC4509F0A7C0809170025B
:102B600040C0C230EDE5DE0709F489C058F4C11554
:102B70008DE5D80709F45AC008F069C08091700249
:102B800082602FC0C236EDE5DE0709F47CC0C63A8C
:102B9000FDE5DF0709F481C0C330DD4509F085C0DC
:102BA00080E06EC080916F0282607DC080916F0274
:102BB00016C080916F02886076C08091700282603A
:102BC0004FC080916F0280626EC080916F028064FE
:102BD0006AC00E94380780916F02806864C0846078
:102BE00062C081603DC080916F028E7F5CC0809129
:102BF0006F028D7F58C080916F0216C08091700265
:102C000018C0809170028D7F2BC080916F028F7EE3
:102C10004AC080916F028F7D46C080916F028F7B8A
:102C200042C080916F02877F8B7F3DC08091700290
:102C30008D7F8E7F15C080916F0282FB222720F945
:102C400091E0922790FB82F990FB83F92CC0809150
:102C50007002982F909591708E7F892B90FB81F94F
:102C60008093700222C00E94380780916F0287FB18
:102C7000222720F991E0922790FB87F914C081E088
:102C80000E94360E12C080916F0284FB222720F929
:102C900091E0922790FB84F906C080916F02982FF3
:102CA000909590FB80F980936F0280916F029091D4
:102CB00070020E94B00D0E94380780E001C081E0E0
:102CC000DF91CF910895893289F1F0F4843171F167
:102CD000B0F4873009F077C081E080930B0184E184
:102CE00080930A018AE0809309018EE180930801B4
:102CF00088E08093050188E28093040164C092EE2D
:102D0000980F9A30F0F05FC0803509F444C028F481
:102D10008F3409F058C08AE03FC0813529F08235F0
:102D200009F051C081E038C08FEF36C080913C027D
:102D3000882379F110923C0210923B0210923A02E1
:102D400042C08D5180933C02833099F038F4813039
:102D500069F08230D9F48AE091E00DC0853099F0B5
:102D600078F0863099F484E091E005C08BE091E042
:102D700002C089E091E090933B0280933A0223C025
:102D800088E091E0F8CF85E091E0F5CF10923C0229
:102D90001AC080E0089586EFE0913A02F0913B027C
:102DA000309789F02081082E000C990B820F911D1D
:102DB0008F3F910519F014F08FEF04C097FF02C008
:102DC000108201C0808381E008950F931F9341E03A
:102DD00050E060E070E08A019B0104C0000F111F09
:102DE000221F331F8A95D2F7C901B8010E949007AC
:102DF0001F910F910C943807482F50E0FA01359736
:102E0000EF33F10508F060C0EE59FF4F0C94BF217D
:102E10000E94340E55C080912902817F8E7F80935D
:102E2000290281E080933D0208950E94820248C0F9
:102E300080912902982F9095917090FB80F9809352
:102E4000290291113DC0897F877F10C0809129029E
:102E500081FB222720F991E0922790FB81F9809352
:102E60002902992369F180912902816080932902C6
:102E700027C08091290282FB222720F991E0922726
:102E800090FB82F9ECCF8091290283FB222720F965
:102E900091E0922790FB83F9E2CF0E94380780915E
:102EA0006F0287FB222720F991E0922790FB87F998
:102EB00080936F0205C0895301C08D510E94E516B1
:102EC00081E0089580E0FACF80E0089580E00895E1
:102ED0000C946617CF93C82F80913D02813069F022
:102EE00038F08230C1F58C2F0E94631681E039C022
:102EF0000E94A90C823289F504C00E94A90C82327A
:102F000061F48C2F0E946817811104C08C2F0E94DD
:102F1000FC161FC081E090E01CC08C2F0E94661739
:102F2000811116C0C43189F058F4CB3089F0C0311A
:102F3000B1F482E080933D0288E30E94631608C0EA
:102F4000C93219F0C83321F00AC010923D0207C0FF
:102F500081E0817006C010923D0280E002C080E0F6
:102F6000F8CFCF910895CF93DF9386319C4541F5FB
:102F7000EB010E94A90C982F8A81209102013091C7
:102F80000301882379F09A7A81E009F480E0809344
:102F90003E02911102C069E201C065E3C9010E94CD
:102FA000A9190AC080913E02811102C069E201C0E4
:102FB00065E3C9010E94B4190E94EB0C80E001C0D6
:102FC00081E0DF91CF9108950F931F93CF93DF930B
:102FD000C42FD22FFC0182818823C9F04093410283
:102FE0000E946C1A9093400280933F0280E28C0F03
:102FF000883008F057C0C77081E001C0880FCA95BB
:10300000EAF7DF91CF911F910F910C949504809175
:103010004102481330C080913F02909140020E94CB
:10302000841A883C910538F510E21D0FCD17B9F0D0
:1030300080E28C0F883040F4C77081E001C0880FB7
:10304000CA95EAF70E949C04183028F581E09D2F6C
:10305000977001C0880F9A95EAF70E949504802F17
:103060000E948C041830F0F4D77081E001C0880F02
:10307000DA95EAF70AC080E28C0F883098F4C770BE
:1030800081E001C0880FCA95EAF7DF91CF911F91C7
:103090000F910C949C04802FDF91CF911F910F9181
:1030A0000C948C04DF91CF911F910F9108950F9391
:1030B0009C01CB01243F4CE5340731F188F4293DD4
:1030C000FCE53F07D9F02A3D4CE5340779F1283D6E
:1030D0003C45A9F506E221EE41EE68ED7CE52BC00A
:1030E000263FFCE53F07E1F0A8F0273F3C4539F5D6
:1030F00007E225EE46EE67EF7CE51DC007E225EE10
:1031000045EE69ED7CE517C006E221EE40EE64EF86
:103110007CE511C007E225EE44EE65EF7CE50BC0CF
:1031200006E221EE42EE66EF7CE505C008E221E012
:1031300045EE6AED7CE50E94E41780E008C0FC01E2
:103140008281882319F01092410201C081E00F9121
:103150000895909385018093840108959093470288
:10316000809346020895E0914602F091470230971D
:1031700021F00190F081E02D099480E00895E09124
:103180004602F0914702309799F0209118012223CE
:1031900059F020916F0227FF07C0DC012C91119696
:1031A0002C93119726E02C930280F381E02D099453
:1031B0000895E0914602F0914702309739F022E0FD
:1031C000DC012C930480F581E02D09940895209171
:1031D0004402309145022817390771F09093450257
:1031E00080934402E0914602F0914702309721F02B
:1031F0000680F781E02D09940895209142023091D4
:1032000043022817390771F09093430280934202DA
:10321000E0914602F0914702309721F00084F18559
:10322000E02D09940895FC013296809118018823BD
:1032300031F080916F0287FF02C09EE101C096E0ED
:1032400080E0915028F021912223D9F38F5FF9CFAC
:103250000895662351F1209118012223E9F020916D
:103260006F0227FF19C0462F4695469546954E3169
:10327000E0F4677021E030E002C0220F331F6A954E
:10328000E2F7FC01E40FF11D828190E0282339234D
:1032900081E0232B69F409C0FC0132960896219144
:1032A000621729F0E817F907D1F780E0089581E067
:1032B00008959C01FC0132969FEF80E041914617F2
:1032C00089F09F3F19F4411101C0982F8F5F86301C
:1032D000A9F79F3F39F0F901E90FF11D97FDFA9524
:1032E0006283089508959C012A5F3F4FFC0142814B
:1032F000461301C01282019682179307B9F7089509
:10330000262F2695269526952E3168F4FC01E20F8E
:10331000F11D677021E030E001C0220F6A95EAF7E5
:103320008281282B22830895262F2695269526957F
:103330002E3170F4FC01E20FF11D677021E030E0E6
:1033400001C0220F6A95EAF7209582812823228303
:10335000089520911801222329F020916F0227FD62
:103360000C9480190C94591920911801222329F0EA
:1033700020916F0227FD0C9494190C9473192091DD
:103380001801FC013296222331F080916F0287FFF1
:1033900002C08EE101C086E0DF011D928A95E9F747
:1033A000089508950C94D11983E0809348020C94F9
:1033B000D219811102C081E001C082E080934802ED
:1033C0000C94D2190C94D91981E0809348020C9482
:1033D000D2190C94E41908950C94EB190C94EC197F
:1033E0000C94EB190C94EB190C94EB19CF930E94ED
:1033F000F2190E94FB110E94F019C0E08C2F0E946C
:103400003311811104C0CF5FC530C1F701C081E025
:10341000CF91089508951F920F920FB60F92112425
:103420008F939F93AF93BF9380914902811113C0F3
:1034300080917B0290917C02A0917D02B0917E02EE
:103440004196A11DB11D80937B0290937C02A093B5
:103450007D02B0937E02BF91AF919F918F910F90AB
:103460000FBE0F901F90189580918302843031F128
:103470000E94E3021092490220E488E190E00FB636
:10348000F894A895809360000FBE2093600083B7E6
:10349000817F846083BF83B7816083BF7894889580
:1034A00083B78E7F83BF0FB6F894A8958091600094
:1034B000886180936000109260000FBE08950E94A2
:1034C00038070C94E70282E084BD93E095BD9AEF43
:1034D00097BD80936E0008952FB7F89480917B027A
:1034E00090917C02A0917D02B0917E022FBF089541
:1034F0002FB7F89460917B0270917C0280917D02DD
:1035000090917E022FBF08959C014FB7F89480914F
:103510007B0290917C02A0917D02B0917E024FBF10
:10352000821B930B089578941F920F920FB60F92FF
:1035300011248F939F93AF93BF9380917B029091BF
:103540007C02A0917D02B0917E020196A11DB11D69
:1035500080937B0290937C02A0937D02B0937E02C5
:10356000BF91AF919F918F910F900FBE0F901F90C1
:10357000189587E797E790930108809300089AE0F1
:1035800088E10FB6F894A895809360000FBE9093E1
:103590006000FFCF80916D020895089522E020938E
:1035A000E9002FEF3091E800215035FD06C035EDE0
:1035B0003A95F1F700002111F5CF2091E80025FFA1
:1035C0000BC040E050E066E070E00E940D1D80916D
:1035D000E8008E778093E8000895CF93DF932091E1
:1035E0001801222339F020916F0227FF03C060E207
:1035F00022E002C068E021E02093E9002FEF309143
:10360000E800215035FD06C035ED3A95F1F7000090
:103610002111F5CF2091E80025FF1DC0EC0180911C
:103620001801811105C040E050E068E070E003C07F
:1036300070E040E050E0CE010E940D1D8091E80056
:103640008E778093E80080E2FE01ADE4B2E0019065
:103650000D928A95E1F7DF91CF91089580934A0208
:1036600070934C0260934B0280918302843001F589
:1036700082E08093E9008FEF9091E800815095FD02
:1036800006C095ED9A95F1F700008111F5CF809174
:10369000E80085FF0DC040E050E063E070E08AE4A0
:1036A00092E00E940D1D8091E8008E778093E800E3
:1036B0000895BC0184E00C942E1BBC0183E00C94A3
:1036C0002E1B80918202811109C00E949E1E0E94C1
:1036D000FB1E8091E20084608093E20008951092C6
:1036E000820208950C94E91960917F0281E06111D2
:1036F00001C080E00C94D4199091830281E0943051
:1037000009F080E060917F020C94D91942E061ECED
:1037100081E00E94171E42E261EC82E00E94171EC7
:103720009091830281E0943009F080E060917F0203
:103730000C94E21980918502833009F461C030F461
:10374000813071F0823009F49AC008958A3009F40A
:1037500086C08B3009F46CC0893009F0A8C020C045
:1037600080918402813A09F0A2C08091E800877FAD
:103770008093E8008091880290918902892B21F43E
:1037800060E28DE492E003C060E080E090E070E0F1
:103790000E94581D8091E8008B778093E80008957F
:1037A00080918402813209F082C0809188029091D8
:1037B0008902029708F07BC08091E800877F8093A0
:1037C000E8008091E80082FD05C0809183028111AC
:1037D000F8CF6DC02091F3008091F20090E0922B21
:1037E000029731F48091F100813011F0863021F49C
:1037F0008091F10080936D028091E8008B7753C037
:1038000080918402813A09F052C08091880290919F
:103810008902892B09F04BC08091E800877F809353
:10382000E8008091E80080FFFCCF8091180136C04D
:10383000809184028132D9F5809188029091890229
:10384000892BA9F58091E800877F8093E8000E948A
:103850004C1E80918602809318010C943807809149
:103860008402813221F58091E800877F8093E8000F
:103870000E944C1E8091870280936E020895809171
:103880008402813AA1F48091E800877F8093E80068
:103890008091E80080FFFCCF80916E028093F10060
:1038A0008091E8008E778093E8000C944C1E089578
:1038B00084B7877F84BF0FB6F894A8958091600085
:1038C000886180936000109260000FBE90E080E8F5
:1038D0000FB6F89480936100909361000FBE0C9432
:1038E000E4190E949E1E0E94FB1EE2EEF0E0808121
:1038F0008460808378940C9490218CE091E00C9407
:10390000AE18809183028530A9F4809183028530BE
:1039100079F40E94341A809181028823B1F30E94C5
:10392000F619882391F30E94F71C0E943807EDCF07
:103930000C945F1A089508950C949E1C292F332728
:1039400023303105C9F060F42130310581F0223097
:10395000310509F044C08BE390E02CE232E043C033
:1039600021323105E1F02232310549F138C082E1DE
:1039700090E027E632E037C099278130910549F081
:1039800028F0029761F5E6EFF1E005C0E8E2F2E029
:1039900002C0E8E0F2E0849190E09F0124C061154C
:1039A000710541F061307105D1F489E090E027E5BF
:1039B00032E019C089E090E02EE332E014C06115D6
:1039C000710541F06130710551F486EB90E029E713
:1039D00032E009C080E490E02FE233E004C080E0F0
:1039E00090E020E030E0FA0131832083089580E107
:1039F00089BD82E189BD09B400FEFDCF8091D80068
:103A00008F7D8093D8008091E00082608093E000F9
:103A10008091E00081FDFCCF0895CF92DF92EF927C
:103A2000FF920F931F93CF93DF93EC018B017A01E9
:103A30000E946B1E811133C0E114F10439F0F701CB
:103A400080819181081B190BC80FD91FC12CD12C63
:103A50000115110519F18091E80085FD16C08091CE
:103A6000E8008E778093E800E114F10449F0F70153
:103A700080819181C80ED91ED182C08285E00FC09D
:103A80000E946B1E882321F30AC089918093F10064
:103A900001501109FFEFCF1ADF0ADACF80E0DF9182
:103AA000CF911F910F91FF90EF90DF90CF900895ED
:103AB00020918A0230918B022617370748F0611552
:103AC000710539F42091E8002E772093E80001C0B9
:103AD000B901FC0120E06115710579F18091830243
:103AE0008823F1F18530F1F18091E80083FD3CC03D
:103AF0008091E80082FD2EC08091E80080FFEBCF2E
:103B00002091F3008091F20090E0922B61157105F5
:103B100051F08830910538F421912093F1006150E3
:103B200071090196F3CF21E0089709F020E0809118
:103B3000E8008E778093E800CECF2111CFCF0AC066
:103B400080918302882361F0853061F08091E800E4
:103B500083FD0AC08091E80082FFF2CF80E00895E3
:103B600082E0089583E0089581E0089520918A021B
:103B700030918B022617370748F06115710539F42B
:103B80002091E8002E772093E80001C0B901FC01E4
:103B900020E06115710591F180918302882309F479
:103BA00040C0853009F43FC08091E80083FD3DC0EE
:103BB0008091E80082FD2FC08091E80080FFE9CF6E
:103BC0002091F3008091F20090E0922B6115710535
:103BD00059F08830910540F424912093F1003196FA
:103BE000615071090196F2CF21E0089709F020E0B9
:103BF0008091E8008E778093E800CBCF2111CCCF65
:103C00000AC080918302882361F0853061F0809141
:103C1000E80083FD0AC08091E80082FFF2CF80E0D7
:103C2000089582E0089583E0089581E00895982F33
:103C3000973068F59093E900981739F07091EC008F
:103C40002091ED005091F00003C0242F762F50E01A
:103C500021FD02C09F5FECCF3091EB003E7F30939F
:103C6000EB003091ED003D7F3093ED003091EB00A3
:103C700031603093EB007093EC002093ED00509393
:103C8000F0002091EE0027FDE5CF80E008958F70D1
:103C90008093E90081E008958091840287FF11C03C
:103CA0008091E80082FD05C0809183028111F8CFE8
:103CB00011C08091E8008B770BC08091830288232C
:103CC00049F08091E80080FFF8CF8091E8008E777E
:103CD0008093E80008952091E4003091E50095E696
:103CE0004091EC00842F817040FF23C08091E80058
:103CF00080FD1DC080918302882399F0853099F062
:103D00008091EB0085FD11C04091E4005091E500E9
:103D10002417350729F3915011F09A01E1CF84E07F
:103D2000089582E0089583E0089581E0089580E099
:103D300008954091E80042FFDDCF08950E940C1FD6
:103D40000E94141FE0EEF0E0808181608083E8ED46
:103D5000F0E080818F77808319BCA7EDB0E08C9173
:103D60008E7F8C9380818F7E808310928202089553
:103D70000F931F93CF93DF930E940C1F0E94141F79
:103D8000C8EDD0E088818F778883888180688883B8
:103D900088818F7D888319BC1092830210927F02E4
:103DA000109281021092800200EE10E0F8018081F2
:103DB0008B7F808388818160888342E060E080E03F
:103DC0000E94171EE1EEF0E080818E7F8083E2EE9C
:103DD000F0E0808181608083808188608083F80149
:103DE00080818E7F8083888180618883DF91CF91FD
:103DF0001F910F910895E8EDF0E080818F7E808320
:103E0000E7EDF0E080818160808384E082BF81E023
:103E1000809382020C94B81EE8EDF0E080818E7FE2
:103E200080831092E20008951092DA001092E1006F
:103E300008951F920F920FB60F9211242F933F9364
:103E40004F935F936F937F938F939F93AF93BF93A2
:103E5000EF93FF938091E10082FF0BC08091E2001D
:103E600082FF07C08091E1008B7F8093E1000E9478
:103E70008F218091DA0080FF1FC08091D80080FFE1
:103E80001BC08091DA008E7F8093DA008091D90088
:103E900080FF0DC080E189BD82E189BD09B400FECB
:103EA000FDCF81E0809383020E94611B05C019BC95
:103EB000109283020E946F1B8091E10080FF19C065
:103EC0008091E20080FF15C08091E2008E7F809398
:103ED000E2008091E20080618093E2008091D8004E
:103EE00080628093D80019BC85E0809383020E9491
:103EF000741B8091E10084FF30C08091E20084FF58
:103F00002CC080E189BD82E189BD09B400FEFDCFEE
:103F10008091D8008F7D8093D8008091E1008F7EC2
:103F20008093E1008091E2008F7E8093E200809197
:103F3000E20081608093E20080917F02882311F08B
:103F400084E007C08091E30087FD02C081E001C0EA
:103F500083E0809383020E947C1B8091E10083FFB9
:103F600029C08091E20083FF25C08091E100877F16
:103F70008093E10082E08093830210927F0280911F
:103F8000E1008E7F8093E1008091E2008E7F80933C
:103F9000E2008091E20080618093E20042E060E014
:103FA00080E00E94171E8091F00088608093F000EE
:103FB0000E94721BFF91EF91BF91AF919F918F91E2
:103FC0007F916F915F914F913F912F910F900FBE15
:103FD0000F901F9018951F920F920FB60F921124F9
:103FE0002F933F934F935F936F937F938F939F9301
:103FF000AF93BF93CF93DF93EF93FF93C091E9000B
:10400000CF708091EC00D82FD17080FDD0E8109255
:10401000E9008091F000877F8093F00078940E94FF
:104020002F201092E9008091F00088608093F000CA
:10403000CD2BCF70C093E900FF91EF91DF91CF912D
:10404000BF91AF919F918F917F916F915F914F91B0
:104050003F912F910F900FBE0F901F9018951F93B7
:10406000CF93DF93CDB7DEB7AA970FB6F894DEBF34
:104070000FBECDBFE4E8F2E08091F100819322E031
:10408000EC38F207C9F70E949A1B8091E80083FF81
:104090002EC18091840290918502492F50E04A30D0
:1040A000510508F024C1FA01EF55FF4F0C94BF21D0
:1040B000803821F0823809F01AC108C0809180024E
:1040C00090918102992389F082600FC080918802CB
:1040D0008F70873008F00BC18093E9008091EB006E
:1040E00085FB882780F91092E9009091E800977F7E
:1040F0009093E8008093F1001092F100D1C0282F36
:104100002D7F09F0F4C0882319F0823061F0EFC0F0
:1041100080918602813009F0EAC0933009F080E096
:10412000809381022EC08091860281112AC08091E5
:1041300088028F702FEF280F263008F0D8C08093A8
:10414000E9002091EB0020FF1CC0933021F4809106
:10415000EB00806214C09091EB0090619093EB00B3
:1041600021E030E0A90102C0440F551F8A95E2F713
:104170004093EA001092EA008091EB0088608093FF
:10418000EB001092E9008091E800877F8093E800BF
:104190000E944C1EACC08111AAC0109186021F77EC
:1041A0008091E3008078812B8093E3008091E80088
:1041B000877F8093E8000E944C1E8091E80080FF7A
:1041C000FCCF8091E30080688093E300111102C06E
:1041D00082E001C083E08093830289C080588230EE
:1041E00008F085C080918602909187028C3D53E053
:1041F000950779F583E08A838AE289834FB7F8943B
:10420000DE01139620E03EE051E2E32FF0E0509310
:104210005700E49120FF03C0E295EF703F5FEF701D
:104220008E2F90E0EA3010F0C79601C0C0968D93B3
:104230009D932F5F243149F74FBF8091E800877F1E
:104240008093E8006AE270E0CE0101960E94581D5A
:1042500016C06091880270918902AE014F5F5F4F76
:104260000E949C1CBC01892B09F441C09091E8007C
:10427000977F9093E80089819A810E94B61D809172
:10428000E8008B778093E80032C0803881F5809118
:10429000E800877F8093E80080917F028093F1009F
:1042A0008091E8008E7772CF811121C080918602C3
:1042B0009091870299270297D4F48091E800877F34
:1042C0008093E8008091860280937F020E944C1EBA
:1042D00080917F02811106C08091E30087FD02C0BA
:1042E00081E001C084E0809383020E94861B80915C
:1042F000E80083FF0AC08091E800877F8093E80090
:104300008091EB0080628093EB00AA960FB6F89440
:10431000DEBF0FBECDBFDF91CF911F9108950895ED
:10432000CF93809183028823A1F0C091E900CF70E0
:104330009091EC00892F817090FD80E8C82B10923D
:10434000E9008091E80083FD0E942F20CF70C09388
:10435000E900CF91089597FB072E16F4009407D03B
:1043600077FD09D00E94C52107FC05D03EF4909549
:1043700081959F4F0895709561957F4F0895EE0F39
:10438000FF1F0590F491E02D0994AA1BBB1B51E17E
:1043900007C0AA1FBB1FA617B70710F0A61BB70BB5
:1043A000881F991F5A95A9F780959095BC01CD015A
:1043B0000895FB01DC0104C08D910190801921F466
:1043C00041505040C8F7881B990B0895F999FECFCA
:1043D00092BD81BDF89A992780B50895A8E1B0E013
:1043E00042E050E00C941A22262FF999FECF92BD9C
:1043F00081BDF89A019700B4021639F01FBA20BDAA
:104400000FB6F894FA9AF99A0FBE08950396272FDB
:104410000E94F5210E94F421252F0E94F521242FCE
:104420000C94F5210196272F0E94F5210C94F4217C
:10443000DC01CB01FC01F999FECF06C0F2BDE1BD64
:10444000F89A319600B40D9241505040B8F7089553
:04445000F894FFCF0E
:10445400C800FA01280850011E0A1401CA1AED1AEC
:10446400CE1A5D1B591BCD1A01E200E900EA00B522
:1044740000B600B700CD008301CC008A01920194FC
:10448400012102230224022502260227022A02B362
:1044940000B4006F007000818283E200E900EA004A
:1044A400B500B600B700CD008301CC008A019201AB
:1044B40094012102230224022502260227022A0251
:1044C400B300B4006F0070008182833133323691BF
:0444D40090946697C3
:00000001FF
